:10000000F9EF0EF000000000D4EF0EF00000000049
:0A0010000000000000000000F3D71C
:1001000081CF03F00001E65305E0C00E0314026E38
:10011000028803D0C00E0314026EE7C000F0003264
:10012000009E0032009E0032009E0032009E0F0EA4
:10013000001602500010016E0F0EE715006E0250FF
:100140000012200E0110816E01C081FF200E0010F0
:10015000816E00C081FF03C081FF9F0E0D6E0D2ECA
:08016000FED7000000001200B0
:100168000001E66B060E016EE4C000F0015004E0E9
:1001780000360090FF0FFBD70050800FE76FE25169
:10018800E727BADF020E0C6E8D0E0D6E0D2EFED710
:0A0198000C2EFCD70000000012003E
:1001A2000001E26BE36BE46BE56BDDDFE06BE16BBF
:1001B200800EE119006E800E005C02E1100EE05D1F
:1001C20025E2800EE119006E800E1D18005C02E12E
:1001D2001C50E05D13E2010EE66FE0C000F0E1C0EA
:1001E20001F0003600900136760E0024E96E000E12
:1001F2000120EA6EEECFE7F082DF05D0010EE66F56
:10020200200EE76F7CDFE04BE12BD2D71C6A1D6A20
:10021200E26BE36B010EE46F000EE56FA4DFE06BAF
:10022200E16B800EE119006E800E005C02E1100E9F
:10023200E05D08E2010EE66F200EE76F60DFE04B43
:10024200E12BEFD7E26BE36B010EE46F000EE56F7B
:040252008ADF12002D
:100256000001E26BE36BE46BE56B83DFDE6BDF6B68
:10026600800EDF19006E800E005C02E1100EDE5D6E
:1002760008E2010EE66F200EE76F3FDFDE4BDF2B55
:10028600EFD7E26BE36B010EE46F000EE56F69DFFB
:10029600DE6BDF6B800EDF19006E800E005C02E104
:1002A600100EDE5D08E2010EE66F200EE76F25DF19
:1002B600DE4BDF2BEFD7E26BE36BE46BE56B51DFD5
:0A02C6001A6A1B6A1C6A1D6A120006
:1002D0000001DE510A0A16E1000E1B1802E1000EB1
:1002E0001A180EE1010E1A6E000E1B6E1C6A1D6AB2
:1002F000E26BE36B010EE46F000EE56F35DF01D0BA
:1003000050DF31D01CC000F01DC001F0003600905D
:100310000136760E0024E16E000E0120E26EDEC092
:10032000E6FF000EE66E1C4A1D2A800E1D18006EA8
:10033000800E005C02E1100E1C5C15E3000E1B1821
:1003400002E1000E1A180EE1010E1A6E000E1B6E6D
:100350001C6A1D6AE26BE36B010EE46F000EE56F31
:0803600003DF01D01EDF1200D3
:1003680010D075DF19D0DDC0DEF0AEDF15D014D0A7
:10037800010EE66FDDC0E7F0BFDEDDC0DEF0A4DF12
:100388000BD00001DD510C0AECE0DD510A0AEBE06C
:0A039800DD510D0AECE0ECD7120075
:1003A2000B6A0A6A096A00500402F4CF09F0F3CF1B
:1003B20008F001500502F4CF0BF0F3CF0AF0005021
:1003C2000502F3500926F4500A22E86A0B22015072
:1003D2000402F3500926F4500A22E86A0B2208C0EC
:1003E20000F009C001F00AC002F00BC003F01200D5
:1003F2000134083609360450085E0550D8A0053C81
:10040200095E003601360F0E0C6E013408360936CD
:10041200045000A006D0085E0550D8A0053C095E35
:1004220005D008260550D8B0053C0926003601360D
:100432000C2EEBD700B006D0045008260550D8B0D9
:08044200053C09260000120030
:10044A000001DB6BDC6B800EDC19006E800E005C39
:10045A0002E1100EDB5D16E2DB51D925E96EDC51B3
:10046A00DA21EA6EEE50000A01E10CD0DB51D925FF
:10047A00E96EDC51DA21EA6EEECFDDF070DFDB4B9C
:06048A00DC2BE1D712009B
:100490000001DA6BDB6B800EDB19006E800E005CF6
:1004A00002E10E0EDA5D23E2DAC000F0DBC001F0FB
:1004B0000A0E046E000E056E74DF4C0E0024F66EFC
:1004C000220E0120F76E000EF86E000E01BEFF0E28
:1004D000F8220900F5CF01F00150D91905E1DAC081
:1004E00000F0DBC001F01200DA4BDB2BD4D7FF0E9B
:0804F000006EFF0E016E120008
:1004F800CBC004F0CCC005F004C002F005C003F086
:10050800044A052ACDC000F0CEC001F00001CD4B51
:10051800CE2B00C0E9FF01C0EAFF02C0E1FF03C023
:10052800E2FFEECFE6FF02C0E9FF03C0EAFFEE52AA
:0E05380001E0E2D7CBC000F0CCC001F0120011
:10054600150E0001D56FCF6BD06B800ED019006EE3
:10055600800E005C02E10D0ECF5DD8B081D0CFC019
:1005660000F0D0C001F00A0E046E000E056E16DF14
:10057600004A012AD80E0024F66E220E0120F76EDC
:10058600000EF86E000E01BEFF0EF8220900F5CF30
:1005960001F0000ECE1902E10150CD195EE1010E07
:1005A600D36F000ED46FD16BD26B800ED219006E52
:1005B600800ECE19005C02E1CD51D15D2FE2D15102
:1005C600CB25E96ED251CC21EA6ECFC000F0D0C067
:1005D60001F00A0E046E000E056EE0DE020E002625
:1005E600000E0122D1510026D2510122D80E00243C
:1005F600F66E220E0120F76E000EF86E000E01BE9A
:10060600FF0EF8220900F5CF01F0EE50011803E0C5
:10061600D36BD46B03D0D14BD22BC7D7000ED419D2
:1006260002E1010ED31919E1CFC000F0D0C001F0EC
:100636000A0E046E000E056EB1DED80E0024F66EAC
:10064600220E0120F76E000EF86E000E01BEFF0EA0
:10065600F8220900F5CFD5F003D0CF4BD02B75D7B4
:06066600D5C000F01200F7
:10066C000450000A08E10550000A05E1FF0E006E77
:10067C007F0E016E12000D6A096A086A01500010A3
:10068C00D8B4000C015005180A6E0ABE0D1E0B6A78
:10069C0005AE05D0041E051E042AD8B4052A01AEE9
:1006AC0005D0001E011E002AD8B4012A01500510E5
:1006BC000A6E0ABE10D097DE0BB020D00DAE000C27
:1006CC00001E011E002AD8B4012A081E091E082A81
:1006DC00D8B4092A000C05AE0DD001BE07D00150CC
:1006EC00096E0050086E016A006AE8D7016A006A58
:1006FC00002A000C011E001E0B2ADDD7082AD8B4D4
:10070C00092A0450085CD8A4D9D70550095CD8A490
:10071C00D5D7096A086A002AD8B4012A01AECED707
:06072C000000FF0C1200AA
:10073200150E0001D56FCF6BD06B800ED019006EF5
:10074200800E005C02E10A0ECF5DD8B081D0CFC02E
:1007520000F0D0C001F00A0E046E000E056E20DE1D
:10076200004A012ADC0E0024F66E230E0120F76EE9
:10077200000EF86E000E01BEFF0EF8220900F5CF42
:1007820001F0000ECE1902E10150CD195EE1010E19
:10079200D36F000ED46FD16BD26B800ED219006E64
:1007A200800ECE19005C02E1CD51D15D2FE2D15114
:1007B200CB25E96ED251CC21EA6ECFC000F0D0C079
:1007C20001F00A0E046E000E056EEADD020E00262E
:1007D200000E0122D1510026D2510122DC0E00244A
:1007E200F66E230E0120F76E000EF86E000E01BEAB
:1007F200FF0EF8220900F5CF01F0EE50011803E0D8
:10080200D36BD46B03D0D14BD22BC7D7000ED419E4
:1008120002E1010ED31919E1CFC000F0D0C001F0FE
:100822000A0E046E000E056EBBDDDC0E0024F66EB1
:10083200230E0120F76E000EF86E000E01BEFF0EB1
:10084200F8220900F5CFD5F003D0CF4BD02B75D7C6
:06085200D5C000F0120009
:10085800CBC004F0CCC005F004C0E9FF05C0EAFF36
:10086800EE5203E0044A052AF7D704C002F005C097
:1008780003F0044A052ACDC000F0CEC001F0000103
:10088800CD4BCE2B00C0E9FF01C0EAFF02C0E1FF5B
:1008980003C0E2FFEECFE6FF02C0E9FF03C0EAFFB4
:1008A800EE5201E0E2D7CBC000F0CCC001F012005C
:1008B800150E0001D56FCF6BD06B800ED019006E6E
:1008C800800E005C02E10E0ECF5DD8B081D0CFC0A3
:1008D80000F0D0C001F00A0E046E000E056E5DDD5A
:1008E800004A012A4C0E0024F66E220E0120F76EF3
:1008F800000EF86E000E01BEFF0EF8220900F5CFBB
:1009080001F0000ECE1902E10150CD195EE1010E91
:10091800D36F000ED46FD16BD26B800ED219006EDC
:10092800800ECE19005C02E1CD51D15D2FE2D1518C
:10093800CB25E96ED251CC21EA6ECFC000F0D0C0F1
:1009480001F00A0E046E000E056E27DD020E002669
:10095800000E0122D1510026D25101224C0E002452
:10096800F66E220E0120F76E000EF86E000E01BE24
:10097800FF0EF8220900F5CF01F0EE50011803E050
:10098800D36BD46B03D0D14BD22BC7D7000ED4195D
:1009980002E1010ED31919E1CFC000F0D0C001F077
:1009A8000A0E046E000E056EF8DC4C0E0024F66E7E
:1009B800220E0120F76E000EF86E000E01BEFF0E2B
:1009C800F8220900F5CFD5F003D0CF4BD02B75D73F
:0609D800D5C000F0120082
:1009DE00300E0001CB5D35E3CB51390832E3486A66
:1009EE00300ECB5D006E00C047F04B6A0A0E00025F
:1009FE00F3CF00F0F4CF01F0020E0026000E01221C
:100A0E00DC0E0024F66E230E0120F76E000EF86E3B
:100A1E00000E01BEFF0EF8220900F5CF00F0000E09
:100A2E00016E17C004F018C005F0B4DC00C049F028
:100A3E0001C04AF0010E5E6E030E4312006A016A97
:100A4E001200610ECB5D05E3CB517A0802E3200E56
:100A5E00CB5F410ECB5D36E3CB514D0833E3010E38
:100A6E00486E410ECB5D006E00C047F04B6A0A0E19
:100A7E000002F3CF00F0F4CF01F0020E0026000EBC
:100A8E000122D80E0024F66E220E0120F76E000E03
:100A9E00F86E000E01BEFF0EF8220900F5CF00F031
:100AAE00000E016E17C004F018C005F073DC00C014
:100ABE0049F001C04AF0010E5E6E030E4312006A49
:100ACE00016A12004E0ECB5D36E3CB515A0833E36A
:100ADE00020E486E4E0ECB5D006E00C047F04B6AA4
:100AEE000A0E0002F3CF00F0F4CF01F0020E002642
:100AFE00000E01225A0E0024F66E230E0120F76E10
:100B0E00000EF86E000E01BEFF0EF8220900F5CFA2
:100B1E0000F0000E016E17C004F018C005F03ADCAC
:100B2E0000C049F001C04AF0010E5E6E030E431282
:100B3E00006A016A1200B00ECB5D36E3CB51DF08BE
:100B4E0033E3040E486EB00ECB5D006E00C047F06E
:100B5E004B6A0A0E0002F3CF00F0F4CF01F0020E42
:100B6E000026000E0122620E0024F66E200E0120D9
:100B7E00F76E000EF86E000E01BEFF0EF822090091
:100B8E00F5CF00F0000E016E17C004F018C005F08E
:100B9E0001DC00C049F001C04AF0010E5E6E030E8A
:100BAE004312006A016A1200CBC0D9F06ADC00C0A1
:100BBE00CCF001C0CDF0FF0E011802E1FF0E0018BF
:100BCE0005E1FF0E006EFF0E016E1200030E486E61
:100BDE00CCC047F04B6A0A0ECC03F3CF00F0F4CF33
:100BEE0001F0020E0026000E01224C0E0024F66EBD
:100BFE00220E0120F76E000EF86E000E01BEFF0EE3
:100C0E00F8220900F5CF00F0000E016E17C004F0B7
:100C1E0018C005F0D1EC01F000C049F001C04AF057
:0E0C2E00010E5E6E030E4312006A016A120090
:100C3C00150E0001D56FCF6BD06B800ED019006EE6
:100C4C00800E005C02E1310ECF5DD8B084D0CFC0F5
:100C5C0000F0D0C001F00A0E046E000E056ED1EC4F
:100C6C0001F0004A012A620E0024F66E200E0120CB
:100C7C00F76E000EF86E000E01BEFF0EF822090092
:100C8C00F5CF01F0000ECE1902E10150CD1960E153
:100C9C00010ED36F000ED46FD16BD26B800ED219B4
:100CAC00006E800ECE19005C02E1CD51D15D30E2B8
:100CBC00D151CB25E96ED251CC21EA6ECFC000F0D8
:100CCC00D0C001F00A0E046E000E056ED1EC01F0DE
:100CDC00020E0026000E0122D1510026D251012213
:100CEC00620E0024F66E200E0120F76E000EF86ED8
:100CFC00000E01BEFF0EF8220900F5CF01F0EE50F8
:100D0C00011803E0D36BD46B03D0D14BD22BC6D7D5
:100D1C00000ED41902E1010ED3191AE1CFC000F074
:100D2C00D0C001F00A0E046E000E056ED1EC01F07D
:100D3C00620E0024F66E200E0120F76E000EF86E87
:100D4C00000E01BEFF0EF8220900F5CFD5F003D03E
:0C0D5C00CF4BD02B72D7D5C000F0120096
:100D6800150E0001D56FCF6BD06B800ED019006EB9
:100D7800800E005C02E10D0ECF5DD8B084D0CFC0EC
:100D880000F0D0C001F00A0E046E000E056ED1EC22
:100D980001F0004A012A5A0E0024F66E230E0120A3
:100DA800F76E000EF86E000E01BEFF0EF822090065
:100DB800F5CF01F0000ECE1902E10150CD1960E126
:100DC800010ED36F000ED46FD16BD26B800ED21987
:100DD800006E800ECE19005C02E1CD51D15D30E28B
:100DE800D151CB25E96ED251CC21EA6ECFC000F0AB
:100DF800D0C001F00A0E046E000E056ED1EC01F0B1
:100E0800020E0026000E0122D1510026D2510122E5
:100E18005A0E0024F66E230E0120F76E000EF86EAF
:100E2800000E01BEFF0EF8220900F5CF01F0EE50CA
:100E3800011803E0D36BD46B03D0D14BD22BC6D7A8
:100E4800000ED41902E1010ED3191AE1CFC000F047
:100E5800D0C001F00A0E046E000E056ED1EC01F050
:100E68005A0E0024F66E230E0120F76E000EF86E5F
:100E7800000E01BEFF0EF8220900F5CFD5F003D011
:0C0E8800CF4BD02B72D7D5C000F0120069
:100E9400440E0001CB6F790ECC6F6E0ECD6F610ED8
:100EA400CE6F200ECF6F430ED06F570ED16F200E32
:100EB400D26F560ED36F310ED46F2E0ED56F320E05
:100EC400D66F0A0ED76FD86B7551000A08E12BEC68
:100ED40001F0CB0ED96F000EDA6F25EC02F0120090
:100EE400530E0001B66F650EB76F640EB86F690ECE
:100EF400B96F6E0EBA6F670EBB6F200EBC6F430ED8
:100F0400BD6F510EBE6F2E0EBF6F2E0EC06F2E0E14
:100F1400C16F0A0EC26FC36B430EC46F510EC56F0F
:100F2400430EC66F510EC76F440EC86F450EC96F8E
:100F3400CA6B2BEC01F0B60ED96F000EDA6F25ECFC
:100F440002F0650ECB6F000ECC6FC40ECD6F000E99
:100F5400CE6F7CEC02F0650ECB6F000ECC6FB4C08C
:100F6400CDF0B5C0CEF076DC650ED96F000EDA6F29
:060F740025EC02F0120062
:100F7A005E50000A01E01200650EE96E000EEA6E8C
:100F8A005F50E926D8B0EA2AEECF01F001C0B4F0EA
:100F9A000150000A04E0100E5F5C01E205D05D6AB0
:100FAA000001756B72DF1200B4C0CBF013DD5F2A4B
:020FBA00120023
:100FBC000001B86BB96BB66BB76B3F50B75D02E114
:100FCC003E50B65D44E2B6C000F0B7C001F000364A
:100FDC00009001361E0E0024E96E000E0120EA6E10
:100FEC00EECFC3F0EECFC4F0B4C000F0B5C001F04A
:100FFC000C0E046E000E056ED1EC01F00A0E046EA0
:10100C00000E056E36EC03F0800E0001C419026E62
:10101C00800E0118025C02E10050C35D09E2BB0EB8
:10102C00B825E16E000EB921E26E010EE66E08D015
:10103C00BB0EB825E16E000EB921E26E030EE66E12
:10104C00B84BB92B020EB627000EB723B6D7BB0E82
:10105C00CB6F000ECC6FB8C0CDF0B9C0CEF099EC10
:10106C0003F000C0BAF0100E8014016E0150000A9B
:10107C002DE0BA51150A0CE1BB0ECB6F000ECC6FF4
:10108C00B8C0CDF0B9C0CEF0A3EC02F000C0BAF0FD
:10109C00BA51150A0BE1BB0ECB6F000ECC6FB8C06A
:1010AC00CDF0B9C0CEF05ADE00C0BAF0BA51150A74
:1010BC000CE1BB0ECB6F000ECC6FB8C0CDF0B9C03D
:1010CC00CEF05CEC04F000C0BAF00ED0BA51150AA8
:1010DC000BE1BB0ECB6F000ECC6FB8C0CDF0B9C01E
:0E10EC00CEF0A6DD00C0BAF0BAC000F01200CF
:1010FA00430E0001B46F610EB56F6C0EB66F6C0EC5
:10110A00B76F200EB86F530EB96F690EBA6F670EBC
:10111A00BB6F6E0EBC6F2E0EBD6F2E0EBE6F2E0EE7
:10112A00BF6F0A0EC06FC16B2BEC01F0B40ED96F02
:0A113A00000EDA6F25EC02F012003F
:10114400B4C0A9FF7F0EA616A69CA680A8CF01F066
:0611540001C000F01200D2
:10115A004E0E0001B66F470EB76F200EB86F430EE2
:10116A00B96F610EBA6F6C0EBB6F6C0EBC6F200E3E
:10117A00BD6F530EBE6F690EBF6F670EC06F6E0EE6
:10118A00C16F210EC26F0A0EC36FC46B2BEC01F044
:10119A00B60ED96F000EDA6F25EC02F0B4C0D9F0A2
:0A11AA00B5C0DAF025EC02F01200E7
:1011B4000001A66BA26BA36BA46BA56B010EA06FC1
:1011C400000EA16F020E3E5C016E000E3F58026ECF
:1011D400A151025C02E1A051015C18E3A0C000F03F
:1011E400A1C001F00036009001361E0E0024D96E15
:1011F400000E0120DA6EDE50A427DE50A523A24B98
:10120400A32B020EA027000EA123DCD7800E006EB4
:10121400800EA319005C02E1A251000847E2A2C0BB
:1012240004F0A3C005F0A4C000F0A5C001F036ECA2
:1012340003F000C0A4F001C0A5F0800E026E800E81
:101244000118025C02E10050320804E2A4C045F037
:10125400A5C046F0010E3E5C036E000E3F58046EBE
:1012640003C000F004C001F00036009001361E0EE9
:101274000024E96E000E0120EA6EEECF03F0EECFFB
:1012840004F045C001F046C002F001360190023678
:101294000250045C02E10150035C07E345C0B4F072
:1012A40046C0B5F089DE00C0A6F081D0010E3E5CD8
:1012B400036E000E3F58046E03C000F004C001F03A
:1012C4000036009001361E0E0024E96E000E012047
:1012D400EA6EEECF03F0EECF04F045C001F046C055
:1012E40002F00136019002360450025C02E1035020
:1012F400015C5DE2100E8014016E0150000A2CE0C6
:10130400020E3E5C036E000E3F58046E03C000F0F4
:1013140004C001F00036009001361E0E0024E96E70
:10132400000E0120EA6EEECF03F0EECF04F045C0CC
:1013340001F046C002F00136019002360250045C0E
:1013440002E10150035C04E30001540EA66F03D0D4
:101354000001450EA66F2BD0020E3E5C036E000EFC
:101364003F58046E03C000F004C001F00036009042
:1013740001361E0E0024E96E000E0120EA6EEECF47
:1013840003F0EECF04F045C001F046C002F0013690
:10139400019002360250045C02E10150035C04E354
:1013A4000001D10EA66F03D00001CD0EA66FA6C01A
:0413B40000F0120033
:1013B800080E4114016E0150000A05E1FF0E405C61
:1013C80001E2402A77D0C80E405C1DE392DE010E90
:1013D8005D6E040E756F5F6A406AA06BA16B800E2C
:1013E800A119006E800E005C02E1070EA05D0AE202
:1013F800650EA025E16E000EA121E26EE66AA04B03
:10140800A12BEDD757D00001A06BA16B800EA119BD
:10141800006E800E005C02E1070EA05D12E2A20ED3
:10142800A025B26F000EA121B36FA0C0B4F086DE74
:10143800B2C0E1FFB3C0E2FF00C0E6FFA04BA12BA2
:10144800E5D7A06BA16B800EA119006E800E005C21
:1014580002E1070EA05D0DE2A20EA025E96E000EC6
:10146800A121EA6EEE50000A01E103D0A04BA12BA6
:10147800EAD7800EA119006E800E005C02E1070E0B
:10148800A05D0CE3050E756FA96BA20EB46F000E7C
:10149800B56F5FDEFF0E196E406A0CD0020E5D6EEE
:1014A800030E756FA20EB46F000EB56F17DD406A9C
:0614B8005F6A5FDD120017
:1014BE00080E4114016E0150000A07E1406A5F6A8E
:0C14CE00010E0001756F010E5D6E120032
:1014DA0019061950000A04E10001756BD6DC5D6A31
:0214EA001200EE
:1014EC00A684A0C0A9FFA1C0A8FF7F0EA616A69C2B
:1014FC00550EA76EAA0EA76EA682A6A201D0FDD786
:02150C001200CB
:0E150E00570E0D6E0D2EFED7000000001200CD
:10151C0081CF02F00001A05305E0C00E0214016E51
:10152C00018803D0C00E0214016E0150A111006E8F
:10153C00200E0010816E00C081FF02C081FF9F0E43
:0C154C000D6E0D2EFED7000000001200F6
:101558009A0E596E1D0E5A6E9C0E5B6E000E5C6ED6
:10156800C80E0001616F1B0E626F000E636F000EE4
:10157800646FDA0E516E1B0E526E000E536E000E23
:10158800546EFF0E556EFF0E566E000E576E000E0F
:10159800586EAC8A900EAB6E948E949C9EAA03D023
:0815A800AECF00F0FBD71200EA
:1015B0000001606B4E6A4F6A080ED56ED10ED76E71
:0C15C0003A0ED66EA00EF26ED58E120010
:1015CC0080504118006E0C0E0014016E0150000A80
:1015DC000DE04450000808E244064450000A03E1C0
:0E15EC000C0E8014416E02D0140E446E1200DC
:1015FA00486A5E6A426A640E456E000E466E436A27
:10160A00196A140E446E640E176E000E186E1200DC
:10161A000900F5CFE6FF0006FBE10106F9E1120039
:10162A00FF0E926E936A946A816A946A826A050EC0
:10163A00C26E0E0EC16EBE0EC06E070EB46E1200E2
:06164A005D6A4C6A12000B
:10165000030E0C6E550E0D6E0D2EFED70C2EFCD704
:1016600000019C6B9D6B800E9D19006E800E005CCE
:1016700002E1030E9C5D07E2A06B030EA16F4EDF3B
:101680009C4B9D2BF0D7A06B020EA16F47DFE66B42
:10169000280EE76F80EC00F0E66B100EE76F80EC31
:1016A00000F0E66B0E0EE76F80EC00F0E66B060EC6
:1016B000E76F80EC00F0E66B010EE76F80EC00F066
:1016C000E66B020EE76F80EC00F01A6A1B6A1C6A78
:1016D0001D6A9C6B9D6B800E9D19006E800E005CD8
:1016E00002E1100E9C5D0AE2650E9C25E16E000E83
:0E16F0009D21E26EE66A9C4B9D2BEDD7120009
:1016FE005E50010A02E1030E431255D10A0E470253
:10170E00F3CF02F0F4CF03F0010E0224006E000EB0
:10171E000320016EDC0E0024F66E230E0120F76E00
:10172E00000EF86E000E01BEFF0EF8220900F5CF76
:10173E009CF0000E00019D6F020E0224006E000E42
:10174E000320016E4B500026000E0122DC0E0024F9
:10175E00F66E230E0120F76E000EF86E000E01BE1F
:10176E00FF0EF8220900F5CF00F0000E016E17C033
:10177E0004F018C005F0D1EC01F000C09EF001C0DD
:10178E009FF025D100010A0E4702F3CF02F0F4CFED
:10179E0003F0010E0224006E000E0320016ED80E1F
:1017AE000024F66E220E0120F76E000EF86E000E6B
:1017BE0001BEFF0EF8220900F5CF9CF0000E9D6FC2
:1017CE00020E0224006E000E0320016E4B50002606
:1017DE00000E0122D80E0024F66E220E0120F76EA6
:1017EE00000EF86E000E01BEFF0EF8220900F5CFB6
:1017FE0000F0000E016E17C004F018C005F0D1EC19
:10180E0001F000C09EF001C09FF0E1D000010A0E71
:10181E004702F3CF02F0F4CF03F0010E0224006E64
:10182E00000E0320016E5A0E0024F66E230E0120C8
:10183E00F76E000EF86E000E01BEFF0EF8220900C4
:10184E00F5CF9CF0000E9D6F020E0224006E000E6E
:10185E000320016E4B500026000E01225A0E00246A
:10186E00F66E230E0120F76E000EF86E000E01BE0E
:10187E00FF0EF8220900F5CF00F0000E016E17C022
:10188E0004F018C005F0D1EC01F000C09EF001C0CC
:10189E009FF09DD000010A0E4702F3CF02F0F4CF65
:1018AE0003F0010E0224006E000E0320016E4C0E9A
:1018BE000024F66E220E0120F76E000EF86E000E5A
:1018CE0001BEFF0EF8220900F5CF9CF0000E9D6FB1
:1018DE00020E0224006E000E0320016E4B500026F5
:1018EE00000E01224C0E0024F66E220E0120F76E21
:1018FE00000EF86E000E01BEFF0EF8220900F5CFA5
:10190E0000F0000E016E17C004F018C005F0D1EC07
:10191E0001F000C09EF001C09FF059D000010A0EE8
:10192E004702F3CF02F0F4CF03F0010E0224006E53
:10193E00000E0320016E620E0024F66E200E0120B2
:10194E00F76E000EF86E000E01BEFF0EF8220900B3
:10195E00F5CF9CF0000E9D6F020E0224006E000E5D
:10196E000320016E4B500026000E0122620E002451
:10197E00F66E200E0120F76E000EF86E000E01BE00
:10198E00FF0EF8220900F5CF00F0000E016E17C011
:10199E0004F018C005F0D1EC01F000C09EF001C0BB
:1019AE009FF015D014D04850000AD8B4A7D648508E
:1019BE00010AD8B4E7D64850020AD8B427D74850FF
:1019CE00030AD8B467D74850040AA8E0EBD7010E33
:1019DE00495E000E4A5A000E4A1802E1000E4918DE
:1019EE0040E135D000014B2A800E006E800E9D190D
:1019FE00005C02E19C514B5C11E317C000F018C073
:101A0E0001F0030E046E000E056ED1EC01F000C065
:101A1E0049F001C04AF0030E5E6E06D017C049F0C1
:101A2E0018C04AF0020E5E6EFC0E43161AD09EC00F
:101A3E0049F09FC04AF0010E5E6E030E431211D0A4
:101A4E005E6AFC0E43160DD0FC0E43160AD05E5095
:101A5E00010AC8E05E50020AEAE05E50030AF0E0B6
:041A6E00F3D7120098
:101A7200C26A070EC012C08E9CC000F000360090F1
:101A8200003600900050C212C28040DDC282C2A263
:101A920001D0FDD7C4CF01F0006AC3500012000E7E
:061AA2000112C2901200C7
:101AA8000CD0829214D0828212D04C2A140E4C5C34
:101AB80002E34C6A82720BD00AD05D50000AF1E052
:101AC8005D50010AF0E05D50020AEFE0F5D7120020
:101AD8003AD0F1DC4CD06CDC4AD0080E4114016ECF
:101AE8000150080A20E10001756B406A4AEC07F0D2
:101AF8005D6A9C6B9D6B800E9D19006E800E005C6C
:101B080002E1070E9C5D0FE29CC0A0F0650E9C25CB
:101B1800E96E000E9D21EA6EEECFA1F0E3DC000134
:101B28009C4B9D2BE8D723D0BDEC07F020D0080EA6
:101B38004114016E0150000A02E1020E756F17D0C0
:101B4800C8DC15D014D000017551000AC2E07551E7
:101B5800010AC1E07551020AC0E07551030AE4E0C8
:101B68007551040AE4E07551050AEAE0EBD7120062
:0A1B78009CC017F09DC018F0120089
:101B8200060E5F5C1FE2410E00019C5D04E39C5166
:101B92005A0801E308D0300E9C5D04E39C513908D9
:101BA20001E301D00FD0650EE16E000EE26E5F50D0
:101BB200E126D8B0E22A9CC0E6FF5F2A9CC0DDF095
:061BC200B4EC01F012007A
:101BC800AECF4DF0ABA202D0AB98AB884DC000F0C1
:021BD8001200F9
:0A1BDA00000E9EBA010E006E12000C
:101BE40000019D6BC9D0040E9C15016E0150000AC2
:101BF40010E1010E3E6E000E3F6E006A016A1E0E79
:101C04000024E16E000E0120E26EE66AE66A010E2F
:101C1400426EBED0040E9C15016E0150000A26E1EE
:101C2400010E3E5C036E000E3F58046E03C000F0CC
:101C340004C001F00036009001361E0E0024026E2E
:101C4400000E0120036E02C0E9FF03C0EAFFEECFDD
:101C540000F0EECF01F0004A012A02C0E1FF03C008
:101C6400E2FF00C0E6FF01C0E6FF23D03E4A3F2A60
:101C7400000E3F5C02E1100E3E5C04E3426A9DC02C
:101C840000F01200010E3E5C036E000E3F58046E1D
:101C940003C000F004C001F00036009001361E0EAF
:101CA4000024E16E000E0120E26EE66AE66A020E8E
:101CB400426E6ED0040E9C15016E0150000A24E1A0
:101CC4003E4A3F2A000E3F5C02E1100E3E5C04E3F4
:101CD400426A9DC000F01200010E3E5C036E000ECD
:101CE4003F58046E03C000F004C001F000360090B9
:101CF40001361E0E0024E16E000E0120E26EE66A3B
:101D0400E66A010E426E36D0010E3E5C036E000E92
:101D14003F58046E03C000F004C001F00036009088
:101D240001361E0E0024026E000E0120036E02C056
:101D3400E9FF03C0EAFFEECF00F0EECF01F0004A66
:101D4400012A02C0E1FF03C0E2FF00C0E6FF01C0B8
:101D5400E6FFDAEC08F000C09DF00050150A05E13A
:101D6400210E00019D6F426A05D000019D51000AB9
:101D740001E0426A0DD00CD04250000AD8B433D7E7
:101D84004250010AD8B446D74250020A93E0F3D72E
:061D94009DC000F01200EA
:0E1D9A00ACB202D00000FCD79CC0ADFF12001E
:101DA80000C016F001C015F0F2A41AD0010E4314B9
:101DB800016E0150010A02E1818C01D0819C020E62
:101DC8004314016E0150020A02E1818E02D07F0E97
:101DD8008116D10ED76E3A0ED66E00016081F2944C
:0A1DE80016C000F015C001F0110054
:101DF2000D0E0B6E2D0E0C6ED70E0D6E0D2EFED728
:101E02000C2EFCD70B2EFAD7000000000001756BD8
:101E1200436A0ADC1CDC18DC330EAF6EAC84ACEC1B
:101E22000AF0D8EC0AF0FDEC0AF080CF41F09C0EEB
:101E32000C6ED70E0D6E0D2EFED70C2EFCD74AEC73
:101E420007F0986B996BFF0E9A6F976B9B6B000173
:101E520060A1E8D060914E4A4F2A0A0E046E000E2D
:101E6200056E4EC000F04FC001F036EC03F008C022
:101E720000F009C001F0000E011802E1000E001886
:101E820002E100016083800E4F18006E800E070A87
:101E9200005C02E1D00E4E5C02E34E6A4F6AE6EC51
:101EA2000AF0B0D02BDCBED097DE005226E08BDEEB
:101EB20000C050F000019B51000A1AE150504B0A39
:101EC2000EE1010E9B6F50C09CF066DF040E000114
:101ED200986F000E996FFF0E9A6F976B08D0505053
:101EE200530A05E1060E756F50C09CF055DF05D010
:101EF2005050000A02E100019B6B040E4114016E76
:101F02000150000A02E1438002D0FE0E431641C096
:101F12009CF067DE00C096F00050000A06E096C012
:101F2200DDF0B4EC01F096C097F00001000E9919B3
:101F320002E1000E981906E19B51010A03E19AC0E1
:101F42009CF02ADF000E0001991902E1040E981993
:101F520008E19B51010A03E197C09CF01DDF0001DB
:101F6200976B9A379A91040E8014016E0150000A01
:101F720001E09A81984B992B800E9919006E800E80
:101F8200005C02E1080E985D02E3986B996B4AD0FF
:101F92005E50000A20E120DE00521CE014DE00C088
:101FA20050F00050000A03E10001756B13D050C0DD
:101FB200CBF0EFEC04F0000E011802E1000E001865
:101FC20009E1060E756F50C0DDF0B4EC01F050C0AF
:101FD2009CF0E2DE02D07FEC0BF024D0040E411420
:101FE200016E0150000A02E1438002D0FE0E431648
:101FF20041C09CF0F6DD00C096F000C09CF0C0DD50
:1020020011D010D000017551030AD8B44BD77551C5
:10201200000AD8B449D77551060ABAE07551040AC4
:10202200DDE0EFD7000160A319D060933CDD000131
:102032009C6B1EDD00C09CF001C09DF000019D3331
:102042009C339D9F9D339C339D9F9D339C339D9FCD
:10205200320E9C27000E9D238EDD3DDDF8D6FFD784
:10206200B0050103030103010000B10503030103ED
:1020720003000000B2020103000000000000B303ED
:102082000101030000000000B40503010303030083
:102092000000B5050103010101000000B6040103BF
:1020A200010100000000B705030103010100000067
:1020B200B8040101010300000000B9040301030395
:1020C20000000000BA040303030300000000BB0584
:1020D2000301030103000000BC0503030103010027
:1020E2000000BD050303030103000000BE05010358
:1020F200030301000000BF0403030301000000000A
:10210200C0020301000000000000C104010103013C
:1021120000000000C2040103030100000000C30527
:102122000103010303010000C405010103010100D1
:102132000000C5030103010000000000C604030102
:10214200030100000000C7040101010100000000BA
:10215200C8040303010300000000C90401010303D2
:1021620000000000CA040301010100000000CB05C9
:102172000303010103000000CC040303010100007A
:102182000000CD010100000000000000CE030301A9
:10219200010000000000CF04030101030000000061
:1021A200D0050101030103000000D101030000007A
:1021B20000000000D2050301010103000000D30565
:1021C2000301010301000000D40301030300000026
:1021D2000000D5050301010303000000D60203033A
:1021E200000000000000D703010101000000000010
:1021F200D8030303010000000000D9050301030313
:1022020001000000DA030303030000000000DB0406
:102212000103010300000000DC03030103000000CE
:102222000000A6040103030300000000DD05010312
:10223200010301000000DE020101000000000000B5
:0A224200DF050101030301000000A5
:10224C002E0601030103010300002C060303010108
:10225C00030300003A0603030301010100003F06DB
:10226C00010103030101000027060103030303011D
:10227C0000002D06030101010103000028050301E4
:10228C0003030100000029060301030301030000FE
:10229C002F0503010103010000003D0503010101AD
:1022AC00030000002B0501030103010000002206BE
:1022BC000103010103010000780403010103000084
:0C22CC00000040060103030103010000B4
:1022D8004102010300000000000042040301010163
:1022E8000000000043040301030100000000440350
:1022F800030101000000000045010100000000008A
:102308000000460401010301000000004703030325
:102318000100000000004804010101010000000064
:10232800490201010000000000004A040103030300
:10233800000000004B0303010300000000004C04F0
:1023480001030101000000004D020303000000002A
:02235800000083
:10235A004E0203010000000000004F0303030300C4
:10236A0000000000500401030301000000005104B2
:10237A0003030103000000005203010301000000EF
:10238A000000530301010100000000005401030092
:10239A0000000000000055030101030000000000D6
:1023AA005604010101030000000057030103030062
:1023BA000000000058040301010300000000590452
:1023CA0003010303000000005A0403030101000093
:0223DA00000001
:1023DC00300503030303030000003105010303036D
:1023EC000300000032050101030303000000330564
:1023FC000101010303000000340501010101030088
:10240C000000350501010101010000003605030142
:10241C000101010000003705030301010100000068
:10242C00380503030301010000003905030303030E
:04243C00010000009B
:0E244000536564696E672043512E2E2E0A00EC
:07244E0043514351444500D6
:0F2455004E472043616C6C205369676E210A006B
:020000040030CA
:0E000000240E1F1EFF8381FF0FC00FE00F4074
:00000001FF
